:100066001201000200000040C0166D2900000102C6
:1000760000010A06000200000040010009022000FB
:1000860001010080320904000002FF00000007059C
:100096000102400000070582020004000902200058
:1000A60001010080320904000002FF00000007057C
:1000B6000102400000070582024000000403090413
:1000C60012035100480059005F00430041004D00F3
:1000D6005300140351004800590035002D00430019
:0600E6004D004F00530025
:040200000202C632FE
:01020B0032C0
:0102130032B8
:01021B0032B0
:0102230032A8
:01022B0032A0
:010233003298
:01023B003290
:010243003288
:01024B003280
:010253003278
:01025B003270
:010263003268
:03026B000204DEAC
:030273000205334E
:03027B0002054930
:0302830002055F12
:03028B00020575F4
:0302930002058BD6
:03029B000205A1B8
:0302A3000205B79A
:0302AB000205CD7C
:0302B3000205E35E
:0302BB000205F940
:0302C30002060F21
:10032B0002032E12033380FEC202C200C201120866
:10033B0003D2E843D82090E65CE0FA443DF0D2AF1C
:10034B00D20D12164090E680E0FA54F7F0538EF877
:10035B00C202120A2D30070512036DC207120DA33C
:10036B0080F390E6B9E0FA24F450030204D5EA2AAC
:10037B002A900380730204880204760204D50204D7
:10038B00760204D50204D50203A40204760204808B
:10039B0002047602047802047690E6BBE0FABA0116
:1003AB00028017BA02028040BA03028067BA0602C3
:1003BB00801FBA070280470204D57A667B0090E65D
:1003CB00B3EBF07A667B007B0090E6B4EAF00204B4
:1003DB00D57A787B0090E6B3EBF07A787B007B00E4
:1003EB0090E6B4EAF00204D590E000E0FAA3E0FB5B
:1003FB0090E6B3F07B0090E6B4EAF00204D590E00F
:10040B0000E0FAA3E0FB90E6B3F07B0090E6B4EAE1
:10041B00F00204D590E6BAE0FA600DBA0102801F33
:10042B00BA020280300204D57AC27B0090E6B3EBAD
:10043B00F07AC27B007B0090E6B4EAF00204D57A36
:10044B00C67B0090E6B3EBF07AC67B007B0090E6B0
:10045B00B4EAF080757AD87B0090E6B3EBF07AD8EB
:10046B007B007B0090E6B4EAF0805F805D758200D4
:10047B00120AC48055758201120AC4804D90E6B8E9
:10048B00E0FABA8002800ABA81028005BA823B8008
:10049B0008900000120AD7803190E6BCE0FA5302B4
:1004AB007E90E6BCE0FBC374809BE433FB4A901662
:1004BB00D593FA3395E0FB74A12AFA74E63BFB74EF
:1004CB00015AF582758300120AD790E6A0E0FA4430
:0304DB0080F0228C
:0A16D50000010202030304040505EE
:1004DE00C0E0C0F0C082C083C002C003C004C0052B
:1004EE00C006C007C000C001C0D075D000120DAE4E
:1004FE009203A203920720030890E6A0E0FA44803C
:10050E00F05391EF90E65D7401F0D0D0D001D000A1
:10051E00D007D006D005D004D003D002D083D0822D
:10052E00D0F0D0E032C0E0C082C0835391EF90E6AD
:10053E005D7402F0D083D082D0E032C0E0C082C0C1
:10054E00835391EF90E65D7404F0D083D082D0E0B7
:10055E0032C0E0C082C0835391EF90E65D7408F024
:10056E00D083D082D0E032C0E0C082C0835391EFFE
:10057E0090E65D7410F0D083D082D0E032C0E0C03F
:10058E0082C0835391EF90E65D7420F0D083D082C9
:10059E00D0E032C0E0C082C0835391EF90E65D742C
:1005AE0040F0D083D082D0E032C0E0C082C083530E
:1005BE0091EF90E65D7480F0D083D082D0E032C0AF
:1005CE00E0C082C0835391EF90E65F7401F0D08358
:1005DE00D082D0E032C0E0C082C0835391EF90E66B
:1005EE005F7402F0D083D082D0E032C0E0C082C00F
:1005FE00835391EF90E65F7404F0D083D082D0E005
:10060E0032C0E0C082C083D20890E68DE4F05391F0
:10061E00EF90E65F7408F0D083D082D0E032C281D2
:10062E0090E6F574FFF000000090E6C07455F000FF
:10063E00000090E6047480F000000090E60474025E
:10064E00F000000090E604E4F000000090E618E4EC
:10065E00F000000090E6CEE4F000000090E038E0FC
:10066E00FA90E6CFF000000090E037E0FA90E6D086
:10067E00F000000090E036E0FA90E6D1F0000000C5
:10068E0075BB0490E032E4F0A3F0A3F0A3F022E5F2
:10069E00BB30E7FB90E6487452F090E618740CF00D
:1006AE00000000D28190E6047480F000000090E615
:1006BE00047402F000000090E604E4F00000002252
:1006CE0090E6F574FFF000000090E6C07455F0005F
:1006DE00000090E6047480F000000090E6047402BE
:1006EE00F000000090E604E4F000000090E618E44C
:1006FE00F000000090E6CEE4F000000090E6CFE4BB
:10070E00F000000090E01FE0FA90E6D0F00000004C
:10071E0090E01EE0FA90E6D1F000000075BB0400F8
:10072E000000E5BB30E7FB90E6487452F090E61807
:10073E00740CF000000090E6047480F0000000904D
:10074E00E6047402F000000090E604E4F0000000FD
:10075E0022C281300B0890E618740DF0800690E6E8
:10076E0018740CF090E6F574FFF000000090E6C0EF
:10077E00E4F000000090E6047480F000000090E6C3
:10078E00047402F000000090E604E4F00000009013
:10079E00E6CEE4F000000090E038E0FA90E6CFF00C
:1007AE0000000090E037E0FA90E6D0F000000090F4
:1007BE00E036E0FA90E6D1F0000000C28C90E03214
:1007CE00E4F0A3F0A3F0A3F0D28C90E6CFE0FA70A1
:1007DE000E90E6D0E0FA700790E6D1E0FA600D7563
:1007EE00BB04000000E5BB20E7E080F990E648740A
:1007FE0002F0D2812290E600E0FA74E75A90E60009
:10080E004410F000000090E60B7401F00000009020
:10081E00E61274E0F000000090E613E4F000000031
:10082E0090E614E4F000000090E615E4F0000000FD
:10083E0090E61074A0F000000090E6D27402F00072
:10084E00000090E6047480F000000090E60474024C
:10085E00F000000090E604E4F000000090E68DE465
:10086E00F090E60174CAF090E6F574FFF090E6F3AE
:10087E0074A0F090E6C37410F090E6C1E4F090E638
:10088E00C2F090E6F4F075AF07759DE4759E007AA0
:10089E00DF7B168B9A7ADF7B167B008A9B90E002B9
:1008AE007440F090E002E0FA1490E002F0EA600B7F
:1008BE0090E67BE0FA90E67CF080E890E6C6E4F005
:1008CE0090E6C7F090E6C8F090E6C9F090E6CAE46C
:1008DE00F090E6CBF090E6CCF090E6CDF090E6808E
:1008EE00E0FA30E70D90009FE4F09000A07402F063
:1008FE00800B90009F7440F09000A0E4F090E6789A
:10090E00E0FA4480F090E67974A0F0120BD690E6EF
:10091E00797405F0120BD690E678E0FA4440F012A6
:10092E000BD690E678E0FA4480F090E67974A1F068
:10093E00120BD690E678E0FA4420F090E679E0FAD1
:10094E00900072F0120BD690E678E0FA4440F01266
:10095E000BD690E679E0FA900072F090E678E0FA25
:10096E004440F090E678E0FA4480F090E67974A086
:10097E00F0120BD690E6797406F0120BD690E6784C
:10098E00E0FA4440F0120BD690E678E0FA4480F09C
:10099E0090E67974A1F0120BD690E678E0FA442036
:1009AE00F090E679E0FA900073F0120BD690E678AC
:1009BE00E0FA4440F0120BD690E679E0FA9000731C
:1009CE00F090E678E0FA4440F09000A0E0FA90E66D
:1009DE0020F000000090009FE0FA90E621F0000069
:1009EE000090E0007482F0A37400F0D20090E671E3
:1009FE00E4F075B40090E670E4F075B2F390E67230
:100A0E00E4F075B60075800375B50075B30090E619
:100A1E0000E0FA4402F090E65EE0FA4408F022C2EA
:100A2E000BC20690E00BE4F0A3F0A3F0A3F0C20912
:100A3E0090E013E4F0A3F0A3F0A3F090E032E4F022
:100A4E00A3F0A3F0A3F0C20A90E03974FFF0A3F074
:100A5E00A374FFF0A3F090E03D74FFF0A3F0A37435
:100A6E00FFF0A3F012145C120A9E90E01BE4F090CB
:0E0A7E00E02EF0A3F0A3F0A3F0C204C2052204
:1016DF0001010101010101070200020002000200E5
:1016EF000100010001000100000000000000003FA8
:1016FF000138010101010107000300000000000093
:10170F000001000000000000002D00000000003F5D
:0C031F00C204C205C208C209C20AC20B17
:100A8C007AFF7BFF8A048B051ABAFF011BEC4D70B1
:100A9C00F322C280120A8CD28090E03274FFF0A351
:100AAC00F0A374FFF0A3747FF090E01D7401F002CA
:020ABC000B56D7
:10171F0000000000000000000000000000000000BA
:0B172F00186AC8FFFFFFFFFFFFFFFF6D
:1000000002033302DEAD00000000000214740000A1
:1000100000000002DEAD000000000002DEAD0000C6
:1000200000000002DEAD000000000002DEAD0000B6
:1000300000000002DEAD000000000002DEAD0000A6
:10004000000000020100000000000002DEAD000020
:10005000000000020100000000000002DEAD000010
:0600600000000002DEAD0D
:100100000204DE00020533000205490002055F001B
:100110000205750002058B000205A1000205B7006B
:100120000205CD000205E3000205F90002060F00FA
:1001300002DEAD0002DEAD0002DEAD0002DEAD008B
:1001400002DEAD0002DEAD0002DEAD0002DEAD007B
:1001500002DEAD0002DEAD0002DEAD0002DEAD006B
:1001600002DEAD0002DEAD0002DEAD0002DEAD005B
:1001700002DEAD0002DEAD0002DEAD0002DEAD004B
:1001800002DEAD0002DEAD0002DEAD0002DEAD003B
:1001900002DEAD0002DEAD0002DEAD0002DEAD002B
:1001A00002DEAD0002DEAD0002DEAD0002DEAD001B
:0801B00002DEAD0002DEAD002D
:100ABE0012062C02069DAA8290E740EAF090E68A82
:100ACE00E4F090E68B7401F022AA82AB838A047D57
:100ADE000090E740ECF08B027B0090E741EAF0904B
:100AEE00E68AE4F090E68B7402F022AA82AB83AC25
:100AFE00F0FD8A067F007800790090E740EEF08BDB
:100B0E00028C038D047D008A067F007800790090A8
:100B1E00E741EEF08B028C038D047D008A067F0088
:100B2E007800790090E742EEF08B028C038D047D05
:100B3E00007B007C007D0090E743EAF090E68AE4BB
:100B4E00F090E68B7404F02290E01DE0FA701C9099
:100B5E00E022E0FAA3E0FBA3E0FCA3E0FD90E017A7
:100B6E00EAF0A3EBF0A3ECF0A3EDF090E01DE0FAB9
:100B7E00BA011190E01774C8F0A3746AF0A3741848
:100B8E00F0A3E4F090E017E0FAA3E0FBA3E0FCA3EF
:100B9E00E0FD8A067F007800790090E036EEF08B5B
:100BAE00028C038D047D008A067F00780079009008
:100BBE00E037EEF08B028C038D047D007B007C0011
:100BCE007D0090E038EAF0227A647B008A048B057F
:100BDE001ABAFF011BEC4D70F322120A9E90E01D13
:100BEE007401F0120B567A407BE78B9A7A407BE7C2
:100BFE007B008A9B12062C90E678E0FA4480F090F7
:100C0E00E67974BAF0120BD690E679742BF0120BCB
:100C1E00D690E67BE0FA90E679F0120BD690E67B62
:100C2E00E0FA90E679F0120BD690E67BE0FA90E6C9
:100C3E0079F0120BD690E67BE0FA90E679F0120B83
:100C4E00D690E67BE0FA90E679F0120BD690E67B32
:100C5E00E0FA90E679F0120BD690E67BE0FA90E699
:100C6E0079F0120BD690E67BE0FA90E679F0120B53
:100C7E00D690E678E0FA4440F0120BD690E678E093
:100C8E00FA4480F090E67974BAF0120BD690E679B9
:100C9E007401F0120BD690E67BE0FA90E679F01232
:100CAE000BD690E67BE0FA90E679F0120BD690E642
:100CBE007BE0FA90E679F0120BD690E67BE0FA90A4
:100CCE00E679F0120BD690E67BE0FA90E679F01218
:100CDE000BD690E67BE0FA90E679F0120BD690E612
:100CEE007BE0FA90E679F0120BD690E67BE0FA9074
:100CFE00E679F0120BD690E678E0FA4440F0120B4B
:100D0E00D690E678E0FA4480F090E67974BAF01264
:100D1E000BD690E6797409F0120BD690E67BE0FACA
:100D2E0090E679F0120BD690E67BE0FA90E679F039
:100D3E00120BD690E678E0FA4440F090E678E0FAAE
:100D4E004480F090E67974BAF0120BD690E679747E
:100D5E0062F0120BD690E679741CF0120BD690E668
:100D6E0079749EF0120BD690E678E0FA4440F012B9
:100D7E00069D90E01DE4F0120B56120ABE90E03272
:100D8E00E0FAA3E0FBA3E0FCA3E0FD90E01BEAF099
:100D9E00E02401F022300A0712075FC20AC20922BC
:100DAE0090E6B9E0FABA10030213A3BA11030210C7
:100DBE0030BA12030211EBBA1303021039BA14033C
:100DCE00021078BA1503021123BA17030210F1BAF2
:100DDE001803021307BA19030212DABA200302101B
:100DEE009ABA2103021335BA220302136CBA2503F1
:100DFE00020FF3BA2603020F7CBA27030210D8BAE9
:100E0E005502800FBA660302110DBA68030211185B
:100E1E0002145390E6BCE0FA603CBA01028051BA6B
:100E2E0002028066BA0302807BBA0403020ECCBAB9
:100E3E000503020EE4BA0603020EFCBA0703020F04
:100E4E0016BA0803020F30BA0903020F48BA630339
:100E5E00020F61020F6F90E017E0FAA3E0FBA3E030
:100E6E00FCA3E0FD8A828B838CF0120AF9021458DF
:100E7E0090E032E0FAA3E0FBA3E0FCA3E0FD8A825F
:100E8E008B838CF0120AF902145890E00BE0FAA34F
:100E9E00E0FBA3E0FCA3E0FD8A828B838CF0120AB8
:100EAE00F902145890E013E0FAA3E0FBA3E0FCA3D0
:100EBE00E0FD8A828B838CF0120AF9021458E4A2A8
:100ECE000933FA7B007C007D008A828B838CF0EDE7
:100EDE00120AF9021458E4A20A33FA7B007C007D50
:100EEE00008A828B838CF0ED120AF902145890E07E
:100EFE0003E0FAA3E0FBA3E0FCA3E0FD8A828B8370
:100F0E008CF0120AF902145890E007E0FAA3E0FB05
:100F1E00A3E0FCA3E0FD8A828B838CF0120AF90217
:100F2E00145890E01BE0FA7B007C007D008A828BD7
:100F3E00838CF0ED120AF902145890E01EE0FAA329
:100F4E00E0FB7C007D008A828B838CF0ED120AF927
:100F5E00021458900009E4F5F07410120AF9021404
:100F6E005890FFFF74FFF5F0120AF902145890E63C
:100F7E0078E0FA4480F090E67974A0F0120BD690E7
:100F8E00E6BCE0FA90E679F0120BD690E678E0FA3D
:100F9E004440F0120BD690E678E0FA4480F090E6EA
:100FAE007974A1F0120BD690E678E0FA4420F09016
:100FBE00E679E0FA90E021F0120BD690E678E0FAAE
:100FCE004440F0120BD690E679E0FA90E740F090AC
:100FDE00E68AE4F090E68B7401F090E678E0FA444D
:100FEE0040F002145890E678E0FA4480F090E679EA
:100FFE0074A0F0120BD690E6BCE0FA90E679F012EF
:10100E000BD690E6BAE0FA90E679F0120BD690E69F
:10101E0078E0FA4440F090E68AE4F090E68BF00235
:10102E00145890DEAD120AD702145820093090E6FB
:10103E00BAE0FAA3E0FBA3E0FCA3E0FD90E022EA15
:10104E00F0A3EBF0A3ECF0A3EDF090E68AE4F090C1
:10105E00E68BF090E6A0E0FA20E1F8120BE890E6BD
:10106E008AE4F090E68BF002145820091390E6BA49
:10107E00E0FAA3E0FB90E01EEAF0A3EBF01206CE3E
:10108E0090E68AE4F090E68BF002145890E6F57440
:10109E00FFF000000090E6487482F090E604748041
:1010AE00F000000090E6047402F000000090E604E8
:1010BE00E4F0000000C209C20A120A9ED28190E634
:1010CE008AE4F090E68BF002145820090DC208D283
:1010DE000A90EEDE120AD702145890DEAD120AD72D
:1010EE00021458200910C208120ABED20A90EEDE6F
:1010FE00120AD702145890DEAD120AD7021458D233
:10110E000B90EEDE120AD7021458C20B90EEDE12CE
:10111E000AD70214583009030211E2C20890E6BA47
:10112E00E0FAA3E0FBA3E0FCA3E0FD90E00FEAF001
:10113E00A3EBF0A3ECF0A3EDF090E60174CAF0126D
:10114E000ABE90E00FE0FAA3E0FBA3E0FCA3E0FDF3
:10115E00C3EA9496EB9400EC9400ED940050089042
:10116E00E60174CAF0800690E601748AF090E032CF
:10117E00E0FAA3E0FBA3E0FCA3E0FD90E00FE0FEAD
:10118E00A3E0FFA3E0F8A3E0F9C3EA9EEB9FEC987F
:10119E00ED994004D20A803390E032E0FAA3E0FBEE
:1011AE00A3E0FCA3E0FD90E00FE0FEA3E0FFA3E0D0
:1011BE00F8A3E0F990E00FEEC39AF0EF9BA3F0E8EE
:1011CE009CA3F0E99DA3F0D206D20990EEDE120A9E
:1011DE00D702145890DEAD120AD702145830090304
:1011EE000212D190E60174CAF0C20890E6BAE0FA93
:1011FE00A3E0FBA3E0FCA3E0FD90E00FEAF0A3EB7D
:10120E00F0A3ECF0A3EDF090E032E0FAA3E0FBA344
:10121E00E0FCA3E0FD90E00FE0FEA3E0FFA3E0F80A
:10122E00A3E0F9C3EE9AEF9BE89CE99D5003120AE6
:10123E00BE90E032E0FAA3E0FBA3E0FCA3E0FD9059
:10124E00E00FE0FEA3E0FFA3E0F8A3E0F9C3EA9EFF
:10125E00EB9FEC98ED994004D20A803390E032E097
:10126E00FAA3E0FBA3E0FCA3E0FD90E00FE0FEA3F9
:10127E00E0FFA3E0F8A3E0F990E00FEEC39AF0EFE1
:10128E009BA3F0E89CA3F0E99DA3F0D206D20990AF
:10129E00E00FE0FAA3E0FBA3E0FCA3E0FDC3EA94B9
:1012AE0096EB9400EC9400ED9400500890E60174D7
:1012BE00CAF0800690E601748AF090EEDE120AD72C
:1012CE0002145890DEAD120AD702145890E6BCE014
:1012DE00FA5302F090E02EEAF0A3E4F0A3F0A3F0AC
:1012EE00746F5580FA90E6BCE0FB74905B4AF58013
:1012FE0090EEDE120AD7021458740F5580FA90E061
:10130E002EE0FBA3E0FCA3E0FDA3E0FEE4FFF8F972
:10131E00EA4203EF4204E84205E942068B8090EE72
:10132E00DE120AD7021458746F5580FA90E02EE040
:10133E00FBA3E0FCA3E0FDA3E0FE5303907C007D45
:10134E00007E00E4FFF8F9EA4203EF4204E84205AA
:10135E00E942068B8090EEDE120AD7021458749F73
:10136E005580FA90E02EE0FBA3E0FCA3E0FDA3E0A5
:10137E00FE5303607C007D007E00E4FFF8F9EA4234
:10138E0003EF4204E84205E942068B8090EEDE123E
:10139E000AD702145890E68AE4F090E68BF090E6B5
:1013AE00A0E0FA20E1F890E740E0FAA3E0FBA3E02A
:1013BE00FCA3E0FD90E003EAF0A3EBF0A3ECF0A3B6
:1013CE00EDF090E744E0FAA3E0FBA3E0FCA3E0FD20
:1013DE0090E007EAF0A3EBF0A3ECF0A3EDF090E0C1
:1013EE0003E0FAA3E0FBA3E0FCA3E0FDBAFF0BBB16
:1013FE00FF08BCFF05BDFF028012D204746F55803A
:10140E00FA90E6BCE0FB74905B4AF58090E007E052
:10141E00FAA3E0FBA3E0FCA3E0FDBAFF0BBBFF08C1
:10142E00BCFF05BDFF028012D205749F5580FA9055
:10143E00E6BCE0FB74605B4AF58090E68AE4F090CF
:10144E00E68BF08005740124FF22E424FF22758CC4
:10145E00D1758A4A74F055894401F589438E08D2B4
:10146E008CD2A9D2AF22C0E0C082C083C002C0031A
:10147E00C004C005C006C007C000C001C0D075D0F2
:10148E0000758CD1758A4A90E032E02401F0A3E019
:10149E003400F0A3E03400F0A3E03400F030041E7A
:1014AE0090E003E0FAA3E0FBA3E0FCA3E0FD90E0F4
:1014BE0026EAF0A3EBF0A3ECF0A3EDF0C2043005A6
:1014CE001E90E007E0FAA3E0FBA3E0FCA3E0FD9092
:1014DE00E02AEAF0A3EBF0A3ECF0A3EDF0C2059046
:1014EE00E026E0FAA3E0FBA3E0FCA3E0FD90E026FB
:1014FE00E024FFFEA3E034FFFFA3E034FFF8A3E0F7
:10150E0034FFF990E026EEF0A3EFF0A3E8F0A3E9A4
:10151E00F0EA4B4C4D702E746F5580FA90E02EE031
:10152E00FBA3E0FCA3E0FDA3E0FE5303907C007D53
:10153E00007E00E4FFF8F9EA4203EF4204E84205B8
:10154E00E942068B8090E02AE0FAA3E0FBA3E0FCE0
:10155E00A3E0FD90E02AE024FFFEA3E034FFFFA30A
:10156E00E034FFF8A3E034FFF990E02AEEF0A3EFA9
:10157E00F0A3E8F0A3E9F0EA4B4C4D702E749F55A2
:10158E0080FA90E02EE0FBA3E0FCA3E0FDA3E0FEDA
:10159E005303607C007D007E00E4FFF8F9EA42030D
:1015AE00EF4204E84205E942068B80100602801CD9
:1015BE0090E00FE0FAA3E0FBA3E0FCA3E0FD90E0D7
:1015CE000BEAF0A3EBF0A3ECF0A3EDF030080B90D8
:1015DE00E00BE4F0A3F0A3F0A3F030093C90E00B95
:1015EE00E0FAA3E0FBA3E0FCA3E0FDEA4B4C4D7058
:1015FE0004D20A802490E00BE024FFFAA3E034FF2B
:10160E00FBA3E034FFFCA3E034FFFD90E00BEAF017
:10161E00A3EBF0A3ECF0A3EDF0D0D0D001D000D02E
:10162E0007D006D005D004D003D002D083D082D00C
:02163E00E03298
:01173A000AA4
:10164000300D0A90E680E0FA440AF0800890E680C7
:10165000E0FA4408F09005DC12167390E65D74FF22
:10166000F090E65F74FFF05391EF90E680E0FA545B
:03167000F7F0226E
:0602F500E478FFF6D8FDDD
:1002D300791CE94400601B7A0190171F782675A0EA
:1002E300E0E493F2A308B8000205A0D9F4DAF275AA
:0202F300A0FF6A
:1002FB007800E84400600A790075A000E4F309D89F
:10030B00FC7826E84400600C790190E000E4F0A34F
:04031B00D8FCD9FA37
:10167300AA82AB8390E600E0FC530418BC0011740B
:10168300012AFCE43BFD8C02C313CA13CAFB80127C
:1016930090E600E0FC530418BC1007EBCA25E0CA2F
:1016A30033FB8A048B051ABAFF011BEC4D600DC096
:0D16B30002C0031216C0D003D00280E62250
:0D02C60075817F1216D1E582600302032EC0
:1016C0007400F58690FDA57C05A3E582458370F93D
:0516D0002275820022DA
:00000001FF
